:02000000801B63
:02000300017684
:02000B00015D95
:02001300016A80
:20001B00215A75812820B20775270A516C01D020B3022122758902758C0675B80275221426
:20003B00118175881075A887D2B74387013000FAC200C2B175264BC2B0D526FDD2B0D2B15A
:20005B0080E8DA0A7A04DB06DC04D20011A532E522B4260274FF04F522800BE52270027457
:20007B002714F522800011A5E52375F06484752104C20231EAE5F075F00A8475210231EA94
:20009B00E5F075210031F5517632C082C083C0E0C0F0E52275F003A4F5F09002A893F52309
:2000BB00E5F0A39304FCE5F0A39304FBD0F0D0E0D083D08222D2B0D2B1D2B75176E5272454
:2000DB00AEFCE43401FD31B6E5272390031D93FCE52723A393FDC2B7C2B1ED75F000D5F08B
:2000FB00FDD5E0F7ECD5E0FDB2B020B20BE5277002741514F52701D020B3DFE527B41402CF
:20011B0074FF04F52701D0C2B5E4F58AF58CF58BF58DD20175890575A88875247A3001172D
:20013B00758800AD8CAC8A31B6E4F58AF58CF58BF58DC20175885043870120B2E0012FD5D9
:20015B00240575247AD201320022D2963163D2973163C2973163C29622C2973163D296313B
:20017B0063D2972292973163D2963163C29622D2973163D2963163A29792D5C296227E08AA
:20019B0033317FDEFB318A2233FD7E08318AA2D533DEF9CD13CD317FD29722790378E851A4
:2001BB000CECA807AC06752106C20231EAAD0079007864510CECAC0675210431EAEC75F04D
:2001DB000A8475210231EAE5F075210031F522200208700474108002D202C0E0316574747A
:2001FB003199E5213199D0E0900297933199317422E4FAFB75F001E9486053ED4C7004FF7E
:20021B00FE8049E9334016C3ED9940117004EC98400BC3E833F8E933F905F080E6C3ED991E
:20023B0040117004EC98400BECC398FCED99FDC3B38001C3EA33FAEB33FBC3E913F9E813AC
:20025B00F8D5F0D9EDFFECFEEBFDEAFCC322C3B3225190E5B044F3B4FFF7227525005190D8
:20027B00D5250122E5B044F3B4FFF35190E5B044F3B4FFE722E40000D5E0FB223F065B4FC6
:20029B00666D7D077F6F777C395E7971002805DC2A05952C05542E05183004E23204B034BD
:2002BB00048236045738042F3A040A3C03E83F03B842038D4503664803414C03155002EE88
:2002DB005402CA5802AA5C028C6002716402586802416C022C7002187402057801F47E012E
:2002FB00DC8401C78A01B39001A198018BA00177A80165B00155B80146C00139C8012CD03D
:20031B0001213E023D023B023A0239023702360235023302320231022F022E022D022C026B
:0C033B002A0229022802270225022402BF
:00000001FF
